:100000008A110A120528000009000730990083169A
:10001000051085100511851505128512831205102E
:100020008510051105128512E830A0000330A100EB
:1000300094213720AC012C08143C031C3328AD015B
:100040002D083B3C031C2D28E830A0000330A10004
:1000500094210130AD07031C20281F308305013097
:10006000AC07031C1B281F308305192836280514EC
:100070009030A0000130A10094218A203421AD20CD
:100080003421CF2034216A203421602034213421CE
:10009000652034215D2034218F20342199203421A2
:1000A0005D203421922034215D2043218021C830FD
:1000B000A000A1019421051008005A216D2108001B
:1000C0006D215A215A215A2108006D215A216D2192
:1000D0005A2108006D215A215A2108005A2108008E
:1000E0005A215A216D215A2108006D216D215A2172
:1000F00008005A215A215A215A2108005A215A210E
:1001000008005A216D216D216D2108006D215A21B1
:100110006D2108005A216D215A215A2108006D21B4
:100120006D2108006D215A2108006D216D216D217E
:1001300008005A216D216D215A2108006D216D2181
:100140005A216D2108005A216D215A2108005A2197
:100150005A215A2108006D2108005A215A216D2187
:1001600008005A215A215A216D2108005A216D2177
:100170006D2108006D215A215A216D2108006D2141
:100180005A216D216D2108006D216D215A215A21BE
:1001900008006D216D216D216D216D2108005A210E
:1001A0006D216D216D216D2108005A215A216D218B
:1001B0006D216D2108005A215A215A216D216D218E
:1001C00008005A215A215A215A216D2108005A212A
:1001D0005A215A215A215A2108006D215A215A21A7
:1001E0005A215A2108006D216D215A215A215A2184
:1001F00008006D216D216D215A215A2108006D21C1
:100200006D216D216D215A2108005A216D215A213D
:100210006D215A216D2108006D216D215A215A212D
:100220006D216D2108005A215A216D216D215A211D
:100230005A2108006D215A215A216D215A210800A6
:100240006D215A215A215A216D2108006D215A2110
:100250005A215A215A216D210800051105165030E6
:10026000A000A10194210800051105165030A0003E
:10027000A10194215030A000A10194215030A00090
:10028000A10194210800051105165030A000A1011C
:1002900094215030A000A10194215030A000A10170
:1002A00094215030A000A10194215030A000A10160
:1002B0009421080005150512053084000230AA00BB
:1002C0000030A0000330A1002E30A2000030A300B7
:1002D000CF21051105162D21080005150512053041
:1002E00084000230AA000030A0000330A100B63024
:1002F000A2000030A300CF21051105162D21080012
:1003000005150512053084000230AA000030A00057
:100310000330A1008A30A2000230A300CF210511D2
:1003200005162D2108009329A00803199F29A6214D
:10033000A003000000000000000000009429A108B4
:1003400003190800A621A103A00394290C30A500DD
:10035000A50BA829000000001230A200A20BB529AD
:10036000B721B721000000000800B721AE290D30E9
:10037000A400A40BB929000008001030A802000155
:10038000031C013EA902031C0800C6290A30A8026A
:100390000001031C013EA902031C0800C6292A080B
:1003A00080042008A8002108A900BD210130A20274
:1003B000031CA3032A0980052008A8002108A9001E
:1003C000BD21A208031DCF29A308031DCF290800C2
:02400E00C431BB
:00000001FF
